:020000040000FA
:100000008BEF00F0F76A140FF66E000EF72209006E
:10001000F550120076616C41444330203D20257537
:100020000D0A0000C150C00B0E09C16EC080C08215
:10003000C084C09EC280C69A949E93809392010E03
:10004000C66E000EC76ED190800ED56ECD6A000EC2
:10005000CA6E000ECB6EB150480BB16E070EB46E77
:100060009250100E006E002EFED70000B450A19CDE
:10007000B56AFF0E926E936E800E946E9EEF00F046
:100080000B50016A0A5C03E20AC000F00CD0006A5F
:10009000080E0C6E0A3600360B50005CD8B0006EAD
:1000A00001360C2EF7D7000C015008C00AF0640E80
:1000B0000B6EE6DF00C008F00150300E07E109A228
:1000C0000DD009B60BD009B8200E03D009960998B7
:1000D0000980012601509EA8FED7AD6E08C00AF027
:1000E0000A0E0B6ECDDF00C008F00150300E06E1A5
:1000F00009B609D009A007D009B8200E0126015081
:100100009EA8FED7AD6E300E082608509EA8FED7DA
:10011000AD6EC1EF00F0F86AD09EEA6AE96AB8965F
:10012000400EAF6EA60EAC6E900EAB6EC150C00B03
:100130000F09C16E070EB46E066A74D794908B9047
:10014000000E016EC250C30B0110C26E100E006E85
:10015000002EFED70000C282C2B2FED7C4CF06F086
:10016000076A07504FDF072A006E00509EA8FED78F
:10017000AD6E0A0E075CF5E106C008F01B0E096EB5
:1001800093D70D0E9EA8FED7AD6E0A0E9EA8FED781
:04019000AD6E03004D
:020000040030CA
:0E0000003FCC390E008781000FC00FE00F408B
:00000001FF
